:030000000236BA0B
:0C36BA0078FFE4F6D8FD75817D02370131
:100E7B0020000A3C2E2E2E3E004950436F6E6E65AD
:100E8B0063745245510A004950436F6E6E6563742B
:100E9B00000A49504E6F41434B210A003E432C56EA
:100EAB002C52432CC0E4E0EFF2E5F020D1E8EDEA60
:100EBB00EEEC49500A003E432C4D41432C25303279
:100ECB0062583A25303262583A25303262583A2508
:100EDB00303262583A25303262583A2530326258F5
:100EEB002C4D414320E0E4F0E5F10A003E432C5643
:100EFB0045522C20332E3220EEF220257320257301
:100F0B002CC2E5F0F1E8FF20495020ECEEE4F3EBC6
:100F1B00FF0A0041707220303320323030390031FB
:100F2B00323A32303A3431003E432C4C442C50523E
:100F3B004F473A2020202020202020202020202036
:100F4B002020202020202020202020202020202096
:100F5B002020202020202020202020202020202086
:100F6B002020202020202020202020202020202076
:100F7B0020202020202020202CC4E0F2E020EFF0C5
:100F8B00EEF8E8E2EAE828F4E0E9EB290A003E2A69
:100F9B002C312CCEF1EDEEE2EDFBE520EFE0F0E0B5
:100FAB00ECE5F2F0FB20F1E5F2E5E2EEE3EE20E812
:100FBB00EDF2E5F0F4E5E9F1E00A003E412C4130B9
:100FCB00312C2562752E2562752E2562752E2562B4
:100FDB00752C495020E0E4F0E5F120E0E4E0EFF27D
:100FEB00E5F0E00A003E412C4130322C2562752E93
:100FFB002562752E2562752E2562752C495020E0D1
:10100B00E4F0E5F120EEF1ED2E20F1E5F0E2E5F074
:10101B00E00A003E412C4130332C2562752E2562AF
:10102B00752E2562752E2562752C495020E0E4F053
:10103B00E5F120F0E5E72E20F1E5F0E2E5F0E00A3E
:10104B00003E412C4130342C2562752E2562752EC5
:10105B002562752E2562752CCCE0F1EAE020F1E5D6
:10106B00F2E80A003E412C4130352C2562752E25C5
:10107B0062752E2562752E2562752CD8EBFEE70A5C
:10108B00003E2A2C312CC4EEEF2E20EFE0F0E0ECEA
:10109B00E5F2F0FB20F1E5F2E5E2EEE3EE20E8ED20
:1010AB00F2E5F0F4E5E9F1E00A003E422C53303171
:1010BB002C2562752CC6E4E0F2FC20E7E0EFF0EEA5
:1010CB00F1E020F1EEE5E4E8EDE5EDE8FF20EEF2EE
:1010DB0020F1E5F0E2E5F0E00A003E422C5330321D
:1010EB002C2562752CCEE1ECE5ED20F120F1E5F03D
:1010FB00E2E5F0EEEC20E1E5E720EAE2E8F2E0EDF4
:10110B00F6E8E90A003E422C5330332C2562752C4D
:10111B00CFE5F0E5E7E0EFF3F1EA20EFF0E820EFC1
:10112B00EEF2E5F0E520F1E2FFE7E820F120F1E552
:10113B00F0E2E5F0EEEC0A003E422C5330352C2564
:10114B0062752CCAE0EDE0EB20F8E8F0EEEAEEE297
:10115B00E5F8E0F2E5EBFCEDEEE3EE20EEE1ECE59D
:10116B00EDE00A003E532C5330362C2530326258BA
:10117B00253032625825303262582530326258257C
:10118B003032625825303262582C4D414320E0E416
:10119B00F0E5F120F8E8F0EEEAEEE2E5F8E0F2E552
:1011AB00EBFCEDEEE3EE20EEE1ECE5EDE00A003ECC
:1011BB00454E440A000A44756D70582020202020AB
:1011CB00303020303120303220303320303420305A
:1011DB003520303620303720303820303920304120
:1011EB002030422030432030442030452030460010
:1011FB000A3A003A20000A000A44756D7044202018
:10120B00202020303020303120303220303320303D
:10121B0034203035203036203037203038203039EC
:10122B0020304120304220304320304420304520B4
:10123B00304600457272206B6579005264206565FB
:10124B0070726F6D0A005264204D454D0A00526456
:10125B0020436F64650A00577269746520436F649D
:10126B00650A0044656275674950204F4E0A004479
:10127B00656275674950204F46460A0044656275A2
:10128B006755736572204F6E0A004465627567552A
:10129B00736572204F46460A0044656275674D734D
:1012AB0067204F6E0A0044656275674D7367204F68
:1012BB0046460A00436F6E666967206C6F636B214D
:1012CB000A00577220656570726F6D0A00205361BA
:1012DB00766520656570726F6D210A00457272200C
:1012EB004D414321004C6F61643E3E002A003C415E
:1012FB0030313D003C4130323D003C4130333D000C
:10130B003C4130343D003C4130353D003C21003CFC
:10131B005330313D003C5330323D003C5330333D74
:0D132B00003C5330353D003C5330363D0052
:064005000113000111008F
:10403B00C28E438910E4F58B758DB8D2ABD28E222C
:03001B0002362A80
:10362A00C0E0C083C082C0D0C28E758B00758DB8D1
:10363A0020170675A61E75A6E10511D213E51360BB
:10364A00020513E512D39401400215120516E51678
:10365A00540F7048D21FE516543F7012D21190666B
:10366A008BE0600A04F0E0D394B44002D21790666B
:10367A0086E0600204F0906104E0600214F0906653
:10368A008CE0D394014003E014F03016020514E5EF
:10369A0015D394644004D21780020515E510D3941B
:1036AA000140021510D28ED0D0D082D083D0E03221
:1008A700C21C7D027C007F07123FE88F4DE54D6437
:1008B7006060097D017F60123F80D21CE4FDFC7FF0
:1008C7000B123FE88F4DE54D30E6097D04E4FF123A
:1008D7003FA4D21C7D017C007F07123FE88F4DE5C6
:1008E7004D7008FD7FFF123F80D21C301C03126041
:1008F70000C288C2A8C2AA75890012358E906349C2
:100907007403F0A374CCF0E4906348F012336A12D6
:100917003ACAC217123CAFD21CC21EC21D906576DE
:100927007408F09062B47424F0E4A3F090633EE09E
:100937009062B6F090633FE09062B7F0906340E05A
:100947009062B8F0906341E09062B9F0906342E042
:100957009062BAF0906343E09062BBF0751201E4D5
:10096700906577F0C218C219C21AC21B201C18AFB3
:100977004DFE7D031230D5E4FF1234347E0E7F7BAB
:10098700E4FBFDFC122CEC90668BE060037401F035
:10099700E4906104F0F514906575F0F51512403B8D
:1009A70075A70775A61E75A6E1D2AFE4F515906188
:1009B70004E0700312133890668CE06401701D9098
:1009C70080007410F09080A874FFF0A3F0A3F0A348
:1009D700F0E490668CF0D21CC21DC21E908008E025
:1009E700F54D30E405D2187410F0E54D30E508D226
:1009F7001A9080087420F0E54D30E608D2199080EF
:100A0700087440F0E514C394034019908002E4F0A1
:100A1700908001F0908000F0E51494064006E4F51C
:100A270014123CAF9080A0E07003123A5C9080B83B
:100A3700E070031239E29080D0E07003123C5390CB
:100A47008000E07013301810122DF3906331EFF02F
:100A5700D394004003120036908002E07006908025
:100A670000E06005D2160209B2C216E4F5149061DF
:100A770004E060030209B2201C12906578E0600C64
:100A87007E0E7F7D122FEDE4906578F0301A1212FA
:100A97002796906331EFF0D394004005E0FF1200F2
:100AA70032201903020C2312260F906331EFF070E6
:100AB700030209B2906375E054BF247F7003020BF1
:100AC7008C147003020B6424026003020BC5201C04
:100AD700077E0E7F84122FED202003020C239063E4
:100AE7004DE0FF7006906351E06061906682E0FE22
:100AF700B50722A3E0FF90634EE0B5071890668420
:100B0700E0FF90634FE0B5070C906685E0FF9063C8
:100B170050E06F6037906351E06E6003020C2390E2
:100B27006683E0FF906352E06F6003020C239066D8
:100B370084E0FF906353E06F6003020C23906685A7
:100B4700E0FF906354E06F6003020C23C2149065CA
:100B5700777401F012409E751201020C2390668B88
:100B6700E060037401F090667AE0FF906377E06FCE
:100B77006003020C2390667AE004F0E4F5129065B6
:100B870075F0020C23301403020C23906344E070C9
:100B9700030209B2906355740AF0123D62D214E45D
:100BA700F512906575F090668604F0E4906679F02A
:100BB700A3F0201C677E0E7F92122FED805E906659
:100BC7008BE060037401F0301452906375E020E706
:100BD7004B906377E0FF906679E0FE6F600D90665B
:100BE70081E07007EE146F70338013906679E0042C
:100BF700F0906331E0FFD3940440031234E4906033
:100C0700007482F0A37401F0906377E0906002F0C3
:100C17007E607F007D031237CD0209B220140302E4
:100C27000D3BE5127068123B35EF60237E647F75DC
:100C3700906476E02404FD1237CD906681E0700958
:100C4700906355E0F5120209B2E4F5120209B29079
:100C57006686E0D3943C4036906681E070309066BB
:100C67008604F0123291E4906475F0A37412F09048
:100C7700667AE0906477F0A374FDF090610563A253
:100C87000190647963A2017F12121FFC809E1240BB
:100C97008C8F4DE54DB401159060007483F0E4A38B
:100CA700F07E607F007D021237CD0209B2E54DD399
:100CB7009401401C9060007483F0A37401F0E54D2B
:100CC70024FEA3F07E607F007D031237CD0209B2B8
:100CD700E512640160030209B2906575E004F02033
:100CE7001C077E0E7F9C122FED906355E0C394C8BE
:100CF7005004E02432F0906575E0C39405400DC2BE
:100D070014E4906577F012409E0209B27C667D82FA
:100D1700906349E0FAA3E0FB7F0212395E7E647FAD
:100D270075906476E02404FD1237CD906355E0F5A5
:100D3700120209B2E512640160030209B2906577F5
:100D4700E014604624FE6042147003020E2E240451
:100D570060030209B2E4F514202013906577740448
:100D6700F0906575E05401F07512010209B29080A8
:100D7700027410F0E4906577F090657504F07512D1
:100D8700FA90668274FFF00209B2906682E07003FF
:100D9700020E189064757480F09064777401F0E423
:100DA700A3F0A304F0A37430F0A3747BF0E4F54D33
:100DB700747C254DF582E43464F583747DF0747D8D
:100DC700254DF582E43464F583E4F0E54D2407907E
:100DD7006476F07C667D82906349E0FAA3E0FB7F4E
:100DE7000212395E7E647F75E54D2409FD1237CD09
:100DF700906681E0601B123D62D214E4F5129065A3
:100E070075F090668604F0E4906679F0A3F0020925
:100E1700B2302007E4906577F08006906577740418
:100E2700F07512FA0209B29080027410F07512057B
:100E3700906575E06401FFF09065777401F0EF70DD
:100E470019906351E06013FCA3E0FDA3E0FEA3E06B
:100E5700FF906682121B8D0209B290634DE0FCA3DE
:100E6700E0FDA3E0FEA3E0FF906682121B8D02095E
:030E7700B280FE48
:010E7A002255
:10003600906376E0B444047F0180027F009063758C
:10004600E0B447047E0180027E00EE5F604A906362
:100056003EE0906377F090633FE0906378F09063C2
:1000660040E0906379F0906341E090637AF09063AA
:1000760042E090637BF0906343E090637CF0906392
:10008600767452F09062AE63A2019080A863A201DA
:100096007F06121FFC02089D906331E0C39408504E
:1000A600030208A690633EE0FF906377E06F60036B
:1000B6000208A690633FE0FF906378E06F6003025A
:1000C60008A6906340E0FF906379E06F6003020842
:1000D600A6906341E0FF90637AE06F60030208A692
:1000E600906342E0FF90637BE06F60030208A69096
:1000F6006343E0FF90637CE06F60030208A69063B1
:1001060076E06444701A9080A8E0B4FF139062AE63
:1001160063A2019080A863A2017F06121FFC8010D3
:100126009062B2E09080ACF09062B3E09080ADF067
:1001360090668BE060037401F090668C7464F090B6
:1001460063767452F0906375E0646D60030202ABEF
:100156007BFF7A0E79A71217197BFF7A0E79C19069
:10016600633EE0F556A3E0F557A3E0F558A3E0F5A6
:1001760059A3E0F55AA3E0F55B1217197556FF75FA
:10018600570F75581E7559FF755A0F755B2A7BFFF9
:100196007A0E79F71217197BFF7A0F79331217192E
:1001A6007BFF7A0F79991217197BFF7A0F79C69020
:1001B6006344E0F556A3E0F557A3E0F558A3E0F550
:1001C600591217197BFF7A0F79F090634DE0F556B7
:1001D600A3E0F557A3E0F558A3E0F5591217197BEC
:1001E600FF7A10791E906351E0F556A3E0F557A308
:1001F600E0F558A3E0F5591217197BFF7A10794CF0
:1002060090633AE0F556A3E0F557A3E0F558A3E06E
:10021600F5591217197BFF7A10796F906336E0F55E
:1002260056A3E0F557A3E0F558A3E0F559121719C0
:100236007BFF7A10798C1217197BFF7A1079B5A299
:1002460020E433F5561217197BFF7A1079E590668C
:1002560081E0F5561217197BFF7A11791090668B9B
:10026600E0F5561217197BFF7A117943A212E4338F
:10027600F5561217197BFF7A11796F90667BE0F5B8
:1002860056A3E0F557A3E0F558A3E0F559A3E0F52A
:100296005AA3E0F55B121719122EF77BFF7A117934
:1002A600BA12171922906375E0644C70737E117F41
:1002B600C0FBFDFC122CEC90637DE0F54EA3E0F54F
:1002C6004FE4F551E54E90637FF0A3E54FF07E11C4
:1002D6007FFB7C637D7F7B02122CECE4F550854F1F
:1002E60082854E83E0FF747F2550F582E43463F502
:1002F60083EFF0054FE54F7002054E0550E550B40B
:1003060010DC7E117FFE7C637D7F7B10122CEC055A
:1003160051E551C3941040AC7E127F01122FED229D
:10032600906375E0646C7060F5527E127F03FBFD8E
:10033600FC122CECE4F551E490637FF0A3E552F057
:100346007E117FFB7C637D7F7B02122CECE4F550F3
:10035600A852E6FF747F2550F582E43463F583EFF7
:10036600F005520550E550B410E67E117FFE7C6321
:100376007D7F7B10122CEC0551E551C3940840B7E4
:100386007E127F01122FED22906375E0644B70613F
:10039600F55074672550F582E43463F583E06032E6
:1003A60074672550F582E43463F583E0F4602374C2
:1003B600672550F582E43463F583E0FF747D2550AC
:1003C600F582E43463F583E0B507100550E550B4D3
:1003D60008C09061047432F002089D906375742120
:1003E600F0301C0302089D7E127F3E122FED02089C
:1003F6009D906375E0B4521A201C077E127F461248
:100406002FED9063757472F07E637F757D081237E9
:100416004622906375E064497045201C077E127F72
:1004260051122FED90637DE0F54EA3E0F54FE4F514
:1004360050854F82854E83E0FF747F2550F582E418
:100446003463F583EFF0054FE54F7002054E055016
:10045600E550B480DC7E637F757D8A123746229034
:100466006375E064437046201C077E127F59122F85
:10047600ED90637DE0F54EA3E0F54FE4F550854F32
:1004860082854E83E493FF747F2550F582E43463BE
:10049600F583EFF0054FE54F7002054E0550E55028
:1004A600B480DB7E637F757D8A1237462290637542
:1004B600E0645A7053201C077E127F62122FED9063
:1004C600637DE0F54EA3E0F54F7C637D7F7B80AFD7
:1004D6004FAE4E123EA6E4F550854F82854E83E41C
:1004E60093FF747F2550F582E43463F583EFF005BE
:1004F6004FE54F7002054E0550E550B480DB7E6334
:100506007F757D8A12374622906375E064446003E6
:1005160002059F90637DE0FF6444700302089DEF2F
:10052600B4310CC21C7E127F6E122FED02089D9014
:10053600637DE0B4300CD21C7E127F7A122FED025E
:10054600089D90637DE0B4320CD21D7E127F871227
:100556002FED02089D90637DE0B4330CC21D7E1220
:100566007F95122FED02089D90637DE0B4340CD286
:100576001E7E127FA4122FED02089D90637DE0B4CB
:10058600350CC21E7E127FB1122FED02089D9063BC
:100596007DE0FF12001E02089D906104E0701320AA
:1005A6001C077E127FBF122FED9063757421F00237
:1005B600089D9061047432F0906375E0FFB45104B5
:1005C600C2AF80FEEF64577045201C077E127FCDB8
:1005D600122FED90637EE0906331F0E4F550906366
:1005E60031E0FFE550C39F400302089D747F25500C
:1005F600F582E43463F583E0FF90637DE0255024C3
:10060600ADF582E43461F583EFF0055080D0906358
:1006160075E0645360030206C1201C077E127FD872
:10062600122FED90633EE0FF9061B6E06F703C9054
:10063600633FE0FF9061B7E06F7030906340E0FF8A
:100646009061B8E0B50724906341E0FF9061B9E09E
:10065600B50718906342E0FF9061BAE0B5070C90C9
:100666006343E0FF9061BBE06F6016906375742191
:10067600F0301C0302089D7E127FE7122FED020860
:100686009DE4F550E4F51574AD2550F582E434612A
:10069600F583E0FDAF50123F060550E550C394FECA
:1006A60040E2C2AFE4907FF0F0A3F0907FFD74AA21
:1006B600F0A374FFF0A37455F080FE906375E064B8
:1006C6004F704C90637DE0F54EA3E0F54FE54F4546
:1006D6004E700A201C077E127FF0122FED201C0799
:1006E6007E127FF7122FEDE4F550747F2550F582C8
:1006F600E43463F583E0854F82854E83F0054FE54C
:100706004F7002054E0550E550B480DE02089D90FC
:100716006375E0FFB4452190637DE0FDA3E0907F23
:10072600F0CDF0A3EDF0C2AF907FFD74AAF0A374F4
:10073600FFF0A37455F080FEEF646560030208A61F
:1007460090637DE0FFA3E0907FF0CFF0A3EFF0E4AD
:10075600F54EF54FD3907FF1E0954F907FF0E09501
:100766004E4021E4F515254FFFE54E3478FE7B809B
:10077600AD4FAC4E123EA67480254FF54FE4354E74
:10078600F54E80D07E127FF9123854EF4E6020125B
:100796000003906344EFF0120003906345EFF012FC
:1007A6000003906346EFF0120003906347EFF07E7C
:1007B600127FFF123854EF4E602012000390634DF3
:1007C600EFF012000390634EEFF012000390634FB8
:1007D600EFF0120003906350EFF07E137F0512389E
:1007E60054EF4E6020120003906351EFF0120003A5
:1007F600906352EFF0120003906353EFF012000380
:10080600906354EFF07E137F0B123854EF4E602046
:1008160012000390633AEFF012000390633BEFF08F
:1008260012000390633CEFF012000390633DEFF07B
:100836007E137F11123854EF4E602012000390632E
:1008460036EFF0120003906337EFF0120003906367
:1008560038EFF0120003906339EFF0E4F550E4F559
:1008660015E55004FF74362550F582E43463F583AC
:10087600E0FD123F060550E550C3944340E0C2AF89
:10088600E4907FF0F0A3F0907FFD74AAF0A374FFCC
:10089600F0A37455F080FE7E637F757D081237469F
:0108A600222F
:103E6E00AE07EEC39430400BEED394395005EE24DA
:103E7E00D0FF22EEC39461400BEED394665005EE54
:103E8E0024A9FF22EEC39441400BEED39446500575
:083E9E00EE24C9FF22AF062249
:104021009062ADE004F070069062ACE004F0906242
:0A403100ACE0FEA3E0FF123DF32215
:10000300124021123E6EEFC454F0FEC0061240218E
:08001300123E6ED0E02FFF2227
:103BF600E4906CC0F0124021906CC1EFF0C3943099
:103C06004018E0FFD394395011906CC0E02405F5BC
:103C160082E43461F583EFF08011906CC0E02405F6
:103C2600F582E43461F583E4F0800C906CC0E00426
:103C3600F0E0D3940840BE755A00755B00755C00D1
:0C3C4600E4F55D7B017A6179051222DC57
:013C5200224F
:043854008E538F54AC
:103858009062ACE4F0A374FFF0124021EF606EF4C4
:10386800606B855482855383E493B507EC755501E5
:10387800E5542555F582E43553F583E493602590A6
:1038880062ADE02555FF9062ACE03400FE123DF3D6
:10389800E5542555F582E43553F583E493B50704DB
:1038A800055580CCE5542555F582E43553F583E478
:1038B8009370A6E55524FFFFE434FFFE9062ADE067
:1038C8002FF09062ACE03EF07E007F0122E4FEFF24
:0138D80022CD
:10336A007E137F17123854EF4E70037F01227E13AB
:10337A007F1A123854EF4E600C124021EF24D024E9
:10338A00FF92208002D2207E137F20123854EF4E03
:10339A00600C124021EF24D0906681F08005E49001
:1033AA006681F07E137F26123854EF4E600C12406D
:1033BA0021EF24D090668BF08005E490668BF07E36
:1033CA00137F2C123854EF4E600C124021EF24D098
:1033DA0024FF92128002C21290633E63A201906699
:1033EA007B63A2017F06121FFC30123B7E137F32E1
:1033FA00123854EF4E603012000390667BEFF012E1
:10340A00000390667CEFF012000390667DEFF012E5
:10341A00000390667EEFF012000390667FEFF012D1
:0A342A000003906680EFF07F00229F
:103DAC00906576E0C3947C503D906576E0FE04F01F
:103DBC0074B42EF582E43462F583EFF0BF0A2790D9
:103DCC006576E0FF04F074B42FF582E43462F58379
:103DDC00E4F0906576E0FF1238D99065767408F0BF
:073DEC009062B5E004F02233
:103CAF009080007480F090633663A201F583F582F3
:103CBF0063A2017F08121FFC90633E63A2019080F4
:103CCF008863A2017F0A121FFC9080927407F0A3F1
:103CDF0074D0F0A37406F0906348E0FF9080B1F0C9
:103CEF009080E1EFF09080957455F0A3F0908000F4
:0A3CFF007401F090800974F0F022C7
:103A5C00908009E04410F09080A0E070609080A10C
:103A6C007482F09080A874FFF0A3F0A3F0A3F07F11
:103A7C00039080AEEFF0A374CBF09080007402F052
:103A8C00906CB0121B9900000000906CB0E090801C
:103A9C0040F0906CB1E0908041F0906CB2E090807E
:103AAC0042F0906CB3E0908043F0A3E4F0A3F0A359
:0D3ABC00F0A3F0908018F0A3F0A3F0A3F0A9
:013AC90022DA
:103C5300908009E04440F09080D17482F07F03901B
:103C630080DEEFF0A374CCF09080027402F0906CCD
:103C7300B4121B9900000000906CB4E0908058F0DF
:103C8300906CB5E0908059F0906CB6E090805AF05B
:103C9300906CB7E090805BF0A3E4F0A3F0A3F0A3F3
:0B3CA300F0908030F0A3F0A3F0A3F03D
:013CAE0022F3
:1039E200908009E04420F09080B8E0706C9080B93B
:1039F2007482F07F039080C6EFF07FCDA3EFF07F5B
:103A0200039080C4EFF0A374CDF09080C074FFF0F7
:103A1200A3F0A3F0A3F09080017402F0906CB812AE
:103A22001B9900000000906CB8E090804CF0906C04
:103A3200B9E090804DF0906CBAE090804EF0906CBE
:103A4200BBE090804FF0A3E4F0A3F0A3F0A3F090CA
:093A52008024F0A3F0A3F0A3F01E
:013A5B002248
:10395E008C4E8D4FA907EAFDE975F018A424ACFF33
:10396E00E5F034808F82F583EDF0EBFDE975F0180C
:10397E00A4FFAEF024ACFBEE34808B82F583A3ED76
:10398E00F0854F828C83E0FDEF24A8FFEE3480FE9D
:10399E008F82F583EDF0854F828C83A3E08F828E2C
:1039AE0083A3F0854F82854E83A3A3E0FDE975F0D6
:1039BE0018A424A8FFE5F03480FE8F82F583A3A31C
:1039CE00EDF0854F828C83A3A3A3E08F828E83A319
:0439DE00A3A3F0228D
:063746008D53AB07AA063B
:10374C00908000E030E5079065787401F022906C71
:10375C00B0E0FCA3E0FDA3E0FEA3E0F5578E568D90
:10376C00558C54AE02AF038E838F8263A201E55653
:10377C00540744C0F58385578263A201AF531220CE
:10378C006EE4FCFDFEE5572553F557EE3556F55620
:10379C00ED3555F555EC3554F554908040E554F025
:1037AC00A3E555F0A3E556F0A3E557F0908000741F
:1037BC0020F0AF57AE56AD55AC54906CB0121B8D7B
:0137CC0022DA
:0637CD008D4EAB07AA06B9
:1037D300908002E030E5079065787403F022906CE6
:1037E300B4E0FCA3E0FDA3E0FEA3E0F5528E518D0F
:1037F300508C4FAE02AF038E838F8263A201E551DB
:10380300540744D0F58385528263A201AF4E122040
:103813006EE4FCFDFEE552254EF552EE3551F551B1
:10382300ED3550F550EC354FF54F908058E54FF09E
:10383300A3E550F0A3E551F0A3E552F090800274A4
:1038430020F0AF52AE51AD50AC4F906CB4121B8D03
:013853002252
:023434008F4EB9
:10343600908001E030E5099065787402F07F002203
:10344600906CB8E0FCA3E0FDA3E0FEA3E0F5528E8D
:10345600518D508C4F90667B63A201E55154074411
:10346600C8F58385528263A2017F06122084E55245
:103476002406F552E43551F551E43550F550E4355E
:103486004FF54F90657963A201E551540744C8F59D
:103496008385528263A201AF4E122084E4FCFDFEB6
:1034A600E552254EF552EE3551F551ED3550F550B4
:1034B600EC354FF54F90804CE54FF0A3E550F0A367
:1034C600E551F0A3E552F09080017420F0AF52AEC2
:0D34D60051AD50AC4F906CB8121B8DAF4E35
:0134E30022C6
:102DF3009081E0E0F54E054E054E054E054E054E1D
:102E0300054E054E054E054E054E908010E0F551DA
:102E1300A3E0F552A3E0F553A3E0F5549081E1E07C
:102E2300F54E054E054E054E054E054E054E054E17
:102E3300054E054E054E908014E0F555A3E0F5567A
:102E4300A3E0F557A3E0F558E557B55308E558B5A2
:102E530054037F0022E4F54EE557540744E0F5831D
:102E630085588263A20190637563A2017F081220D3
:102E7300B490637763A2019062AE63A2017F0612EE
:102E83001FFC906375E0F54FA3E0F550E4F54E9019
:102E93006375E0702AA3E024F8F54EE55754074420
:102EA300E0F58385588274082582F582E43583F53D
:102EB3008363A20190637563A201AF4E1220B4AE87
:102EC3004FE4FCFDE5582550F558E5573EF557ED21
:102ED3003556F556EC3555F555908014E555F0A368
:102EE300E556F0A3E557F0A3E558F0908000744051
:032EF300F0AF4EEF
:012EF60022B9
:10260F009081E6E0F54E054E054E054E054E054E02
:10261F00054E054E054E054E054E908028E0F551AE
:10262F00A3E0F552A3E0F553A3E0F5549081E7E062
:10263F00F54E054E054E054E054E054E054E054E03
:10264F00054E054E054E90802CE0F555A3E0F5564E
:10265F00A3E0F557A3E0F558E4F54EE557B5530A57
:10266F00E558B55405C21902277BE557540744F0C6
:10267F00F58385588263A20190637563A2017F0879
:10268F001220B4906375E0F54FA3E0F550E5504587
:10269F004F70099080027410F07F0022906682E0E4
:1026AF00FFF46030906377E06F600302274290661B
:1026BF0083E0FF906378E06F7079906684E0FF901D
:1026CF006379E06F706D906685E0FF90637AE06FDD
:1026DF006031805F906377E0906682F0906378E07E
:1026EF00906683F0906379E0906684F090637AE06F
:1026FF00906685F090637BE0FFA3E0906349CFF095
:10270F00A3EFF0906375E0702AA3E024F8F54EE58F
:10271F0057540744F0F58385588274082582F58253
:10272F00E43583F58363A20190637563A201AF4E15
:10273F001220B4AE4FE4FCFDE5582550F558E5578F
:10274F003EF557ED3556F556EC3555F555AF54AEBC
:10275F0053AD52AC51AB58AA57A956A855D3121B1B
:10276F006940099080027410F07F002290802CE560
:10277F0055F0A3E556F0A3E557F0A3E558F0908088
:06278F00027440F0AF4EA1
:012795002221
:102796009081E3E0F54E054E054E054E054E054E7D
:1027A600054E054E054E054E054E90801CE0F55132
:1027B600A3E0F552A3E0F553A3E0F5549081E4E0DD
:1027C600F54E054E054E054E054E054E054E054E7B
:1027D600054E054E054E908020E0F555A3E0F556D2
:1027E600A3E0F557A3E0F558E4F54EE557B5530ACF
:1027F600E558B55405C21A0228ECE557540744E8D3
:10280600F58385588263A20190600463A2017F0E5E
:102816001220CA906004E0F54FA3E0F55090600CDA
:10282600E0FFF4604A90667BE0FEEF6E7079A3E00D
:10283600FF90600DE06F706F90667DE0FF90600E18
:10284600E06F706390667EE0FF90600FE06F7057F8
:1028560090667FE0FF906010E06F704B906680E0BE
:10286600FF906011E06F703FE4906013F080089075
:10287600601374FFF0D2D9906004E0702AA3E024BC
:10288600F2F54EE557540744E8F583855882740EF1
:102896002582F582E43583F58363A20190600463A3
:1028A600A201AF4E1220CAAE4FE4FCFDE5582550FA
:1028B600F558E5573EF557ED3556F556EC3555F5D1
:1028C60055AF54AE53AD52AC51AB58AA57A956A802
:1028D60055D3121B695006E550454F70099080018B
:1028E6007410F07F0022908020E555F0A3E556F0A5
:1028F600A3E557F0A3E558F09080017440F0AF4E81
:0129060022AE
:042FED008E538F541C
:102FF100908000E030E5079065787401F022906CD4
:10300100B0E0FCA3E0FDA3E0FEA3E0F55A8E598DEC
:10301100588C57E55AFFE5595407FEE42FF556EE53
:1030210034C0F555855682F5837423F00556E5566F
:10303100700205555355C7F582855583740AF0050D
:1030410056E556700205555355C790633E63A2017C
:1030510085558385568263A2017F0612206E740610
:103061002556F556E43555F55585538385548263C8
:10307100A20185558385568263A201122052E4FC88
:10308100FDFE906CB0E0F8A3E0F9A3E0FAA3E02F15
:10309100FFEE3AFEED39FDEC38FCEF2408FFE43E8B
:1030A100FEE43DFDE43CFC906CB0121B8D906CB0D5
:1030B100E0908040F0906CB1E0908041F0906CB273
:1030C100E0908042F0906CB3E0908043F0908000FB
:0330D1007420F078
:0130D40022D9
:0A2CEC008E538F548C558D568B5774
:102CF600908000E030E5079065787401F022906CD2
:102D0600B0E0FCA3E0FDA3E0FEA3E0F55D8E5C8DE4
:102D16005B8C5AE55DFFE55C5407FEE42FF559EE42
:102D260034C0F558855982F5837423F00559E55961
:102D3600700205585358C7F582855883740AF00502
:102D460059E559700205585358C790633E63A2016E
:102D560085588385598263A2017F0612206E740608
:102D66002559F559E43558F55885538385548263BA
:102D7600A20185588385598263A2011220528F5E73
:102D8600EF2559F559E43558F558E5576017855537
:102D96008385568263A20185588385598263A20181
:102DA600AF5712206EE55E24082557F557FFE4FC61
:102DB600FDFEE55D2FF55DEE355CF55CED355BF50D
:102DC6005BEC355AF55A908040E55AF0A3E55BF086
:102DD600A3E55CF0A3E55DF09080007420F0AF5DA4
:0C2DE600AE5CAD5BAC5A906CB0121B8D63
:012DF20022BE
:0631B6008E4E8F4F8D507C
:1031BC00908000E030E5079065787401F022906C07
:1031CC00B0E0FCA3E0FDA3E0FEA3E0F5568E558D28
:1031DC00548C53E556FFE5555407FEE42FF552EE9B
:1031EC0034C0F551855282F5837423F00552E552B3
:1031FC00700205515351C7F582855183EBF005528E
:10320C00E552700205515351C790633E63A201858C
:10321C00518385528263A2017F0612206E740625AB
:10322C0052F552E43551F551854E83854F8263A298
:10323C000185518385528263A201AF5012206E74B6
:10324C00082550F550FFE4FCFDFEE5562FF556EE33
:10325C003555F555ED3554F554EC3553F553908003
:10326C0040E553F0A3E554F0A3E555F0A3E556F083
:10327C009080007420F0AF56AE55AD54AC53906CAA
:04328C00B0121B8DD4
:01329000221B
:0238D9008F67F7
:1038DB00908000E030E5079065787401F022906CE1
:1038EB00B0E0FCA3E0FDA3E0FEA3E0F56B8E6A8DD8
:1038FB00698C68E56BFFE56A5407FEE42FFFEE3435
:10390B00C09062B463A201F5838F8263A201AF679B
:10391B0012206EE4FCFDFEE56B2567F56BEE356A58
:10392B00F56AED3569F569EC3568F568908040E529
:10393B0068F0A3E569F0A3E56AF0A3E56BF090806E
:10394B00007420F0AF6BAE6AAD69AC68906CB012CE
:02395B001B8DC2
:01395D002247
:0630D5008E4E8F4FAB058B
:1030DB00908000E030E5079065787401F022906CE9
:1030EB00B0E0FCA3E0FDA3E0FEA3E0F5558E548D0C
:1030FB00538C52E555FFE5545407FEE42FF551EE82
:10310B0034C0F550855182F5837423F00551E55198
:10311B00700205505350C7F582855083EBF0055173
:10312B00E5517002055090633E63A2018550838583
:10313B00518263A2017F0612206E74062551F55150
:10314B00E43550F5505350C7E54E85518285508379
:10315B00F00551E551700205505350C7F58285506B
:10316B0083E54FF00551E551700205505350C7E50B
:10317B0055240AF555E43554F554E43553F553E429
:10318B003552F552908040E552F0A3E553F0A3E59C
:10319B0054F0A3E555F09080007420F0AF55AE5479
:0A31AB00AD53AC52906CB0121B8DB6
:0131B50022F7
:0A408100E4FEEEC39F50030E80F82A
:01408B002212
:10358E00E4F54EE54E2401FFE433FE123DF37436AE
:10359E00254EF582E43463F583EFF0054EE54EC318
:1035AE00943F40DFE4F54EE54E247FFFE433FE12F8
:1035BE003DF3742D254EF582E43461F583EFF074FE
:1035CE002D254EF582E43461F583E0FF6003B4FFF0
:1035DE001D742D254EF582E43461F5837420F0744C
:1035EE002E254EF582E43461F583E4F08009054E14
:1035FE00E54EC3948040B0E49061ACF0F54EAF4E12
:10360E007E00123DF374AD254EF582E43461F583F0
:0B361E00EFF0054EE54EC394FE40E3C4
:01362900227E
:103FC800E4FDFCC3ED9FEC9E5015E4FBFA0BBB002F
:0F3FD800010ABA01F8BB90F50DBD00010C80E4A1
:013FE70022B7
:0D405A004390014390025390FE5390FD22CD
:0D4067005390FD5390FE43900243900122C0
:0E404B005390FD439002E5905408FF5390FD02
:014059002244
:0D4074005390FD4390014390025390FD22B4
:07409700AE071FEE70FA22D4
:023EDA00AD0732
:103EDC00E4FC5390FDEDA804088002C333D8FC30F9
:103EEC00E70543900180035390FE7F0512409743F2
:093EFC0090020CBC08DC5390FD9F
:013F05002299
:103F3000E4FF5390FD7E07439002E59030E00D745E
:103F400001A806088002C333D8FC42075390FD1E27
:083F5000C3EE6480948050DF91
:013F58002246
:103F0600AB05AA0712405A7FA0123EDA12404BAF09
:103F160002123EDA12404BAF03123EDA12404B1247
:0A3F260040677F0A7E00123FC822A8
:043DF300AB07AA066A
:103DF700C3EB94FFEA9400400DE42BF58274773A05
:103E0700F583E493FF2212405A7FA0123EDA124054
:103E17004BAF03123EDA12404B12405A7FA1123EBB
:0D3E2700DA12404B123F3012407412406717
:013E3400226B
:023EA6008B533C
:103EA800A2AF9221C2AF85A25453A2FE8E838F8205
:103EB80005A28C838D8274091220F8E55353A2FE63
:103EC80043A2201220FA53A2DF8554A2A22192AF66
:013ED800FFEA
:013ED90022C6
:103FE800A2AF9221C2AF8C838D82EF1220F843A238
:0C3FF800201220FA53A2DFA22192AFFF9A
:014004002299
:023F80008F4E62
:103F8200A2AF9221C2AFE4F5838D8274061220F8AB
:103F9200E54E43A2201220FA53A2DFA22192AF7F64
:013FA200011D
:013FA30022FB
:023FA4008F4E3E
:103FA600A2AF9221C2AFE4F5838D82740A1220F883
:103FB600E54E43A2201220FA53A2DFA22192AF7F40
:013FC60001F9
:013FC70022D7
:101F2100A907E7FFA805EF93C3966008403B74FC3F
:101F31002FFF80F00F08EF93C3966008402B74FBCE
:101F41002FFF80E00F08EF93C3966008401B74FADF
:101F51002FFF80D00F08EF93D3966008400B74F9E0
:101F61002FFF80C01F1F1F1F1FEF54FEF80303F731
:101F7100E893FC08E893FD08E893FE08E893FF2244
:101F810009E993C39D6008402974FB29F980F1098F
:101F9100E993C39E6008401A74FA29F980E209E9BD
:101FA10093D39F6008400B74F929F980D31919194B
:101FB1001919E9C313C313FF22740093F8ECC398F2
:101FC1004024701F740193F8EDC398401970147484
:0E1FD1000293F8EEC398400E7009740393F863
:101FDF00EFC39840037F00227F0122EDF8E6F0085F
:101FEF00A3DFFA22EDF8E0F608A3DFFA22E0A363FD
:101FFF00A201F0A363A201DFF475A2002263A20184
:10200F00F0A363A20122E0A363A201F0A363A201E4
:10201F00E0A363A201F0A363A201E463A201F0A312
:10202F0063A201DFE175A20022E0A363A2016DFEAE
:10203F00936CFDEE058393FC158363A201DFEA75B4
:10204F00A200227F00E493A363A201F00F600CA310
:10205F00E583C2E3F58363A20180EA75A20022E063
:10206F00A363A201F0A3E583C2E3F58363A201DFBB
:10207F00EE75A20022E0A363A201F0A3E583C2E400
:10208F00D2E3F58363A201DFEC75A20022E0A36324
:10209F00A201F0A3E58344F8C2E5F58363A201DF53
:1020AF00EC75A20022E583C2E3F583E0A363A201EE
:1020BF00F0A363A201DFEE75A20022E583C2E4D292
:0A20CF00E3F583E0A363A201F0A390
:1020D90063A201DFEC75A20022E58344F8F583E0F1
:1020E900A363A201F0A363A201DFEE75A20022F9A6
:1020F90022C002C004C00612FFF0D006D004D002EC
:0121090022B3
:10001E00BF360BD207E4F526F527F546F547BF3771
:04002E0002C20722E1
:103B9800C2A9438902906CABE0FFF58C8F8A75D976
:103BA8000475DA4875DB3175DC4975DD4975DE3138
:103BB800E4F5E9F5F9F5EBF5FB906CA9E06016750D
:103BC800EC1075ED10E4F5FCF5FD754208753C1038
:103BD800754101801375EC8075ED80E4F5FCF5FD09
:0E3BE800754280F53C754110E4F5EEF5FE22C5
:103E3500E4FEAF8CEFFD906CAAE07003A3E06D602B
:103E450005123B987E01E5D920E2057E02123B98DA
:103E5500E58920E105123B987E03D28C75D8407523
:083E6500B740D2AED2AFAF06A8
:013E6D002232
:0300330002210A9D
:0D210A00C0E0C0F0C083C082C0D075D00816
:10211700C2AF30DC56C3E5EC95EEC395425012E5ED
:102127004125ECF5EC30D70405FC801685FCFC80D6
:1021370011C3E5EC9541F5EC30D70415FC80038518
:10214700FCFC300724852782852683E590F0052748
:10215700E52770020526F582852683E5EEF005273B
:10216700E5277002052653260FC2DC30D929300730
:1021770024852782852683E590F00527E5277002C9
:102187000526F582852683E5EBF00527E52770020E
:10219700052653260FC2D920DA0302225BE53C70DD
:1021A7000405FC8010E53C25ECF5EC30D70405FC74
:1021B700800385FCFC200803022259302A41AF40E6
:1021C700AE3FAD3EAC3D7801121B7A8F408E3F8DFE
:1021D7003E8C3D309712E540F540E53FF53FE53E43
:1021E700F53EE53D4480F53D200627E540F540E511
:1021F7003FF53FE53EF53EE53D6480F53D8013E55F
:1022070028C313F5283097042480F5282006036394
:102217002880302A23E4FFE53FFEE53EFDE53DFC4F
:10222700AB4BAA4AA949A848C3121B697024F543B6
:10223700F53AF528C22A801A0543E5435407701278
:1022470053433FE543131313541F242AF8A6287555
:102257002800C2DA30DB71E53C700405FD8010E52B
:102267003C25EDF5ED30D70405FD800385FDFDE543
:1022770044653B6029E53B54077013E53B13131393
:10228700541F2432F8E6F5292004036329FFE529C2
:10229700139296E529C313F529053B533B3FB292A9
:1022A700300723852782852683E590F00527E527D4
:1022B70070020526F582852683E4F00527E5277059
:0A22C70002052653260FC2DBD2AF3A
:0B22D100D0D0D082D083D0F0D0E0321B
:101CB9004241554400494E565F52454300494E56EC
:101CC9005F5452414E5300494E565F414C4C0044BB
:101CD9004543495F56414C00003E2A2C312CCFE048
:101CE900F0E0ECE5F2F0FB20F1E8EDF5F0EEEDEDDA
:101CF900EEE3EE20EFEEF0F2E00A003E4C2C42302B
:101D0900312C256C752CD1EAEEF0EEF1F2FC20EEC7
:101D1900E1ECE5EDE02C35302C3130302C3230302F
:101D29002C3330302C3630302C313230302C3234A8
:101D390030302C343830300A003E422C4731302CB8
:101D49002562752CC8EDE2E5F0F1E8FF20EDE02011
:101D5900EFF0E8B8ECE50A003E422C4731312C257A
:101D690062752CC8EDE2E5F0F1E8FF20EDE020EF27
:101D7900E5F0E5E4E0F7E50A003E422C4730322C75
:101D89002562752CD3EFF0E0E2EBE5EDE8E520EF15
:101D9900EEF2EEEAEEEC2020285254532D43545330
:101DA900290A003E532C4730332C256C752CC7E08B
:101DB900E4E5F0E6EAE020F1F2E0F0F2E020EFE518
:101DC900F0E5E4E0F7E828ECF1290A003E532C4756
:101DD90030332C256C752C202AE7E0E4E5F0E6EA9F
:101DE900E020F1F2E0F0F2E020EFE5F0E5E4E0F7E1
:101DF900E828ECF1290A003E2A2C312CC0E4E0EF56
:101E0900F2E5F020F1E8EDF5F0EEEDEDEEE3EE2090
:101E1900EAE0EDE0EBE02E20CFF0EEF2EEEAEEEBB9
:101E290020D0CFD22D383028C0E8F1F2290A003E5F
:101E3900532C5230312C256C752CCFE0F0E0ECE5B9
:101E4900F2F0FB20EFF0EEF0E5E6E8E2E0EDE8FF86
:101E590020D6C1C80A003C21003C4230313D003C3B
:101E69004731303D003C4731313D003C4730323D40
:101E7900003C4730333D003C5230313D000A456D4E
:101E89007074792120000A54726961646520200008
:101E99000A526563206572726F7221000A52656386
:101EA9002064617461000A5265632042434921003C
:101EB9000A526563656976656420466C616721200D
:101EC900000A5472616E736D697420000A000A5425
:101ED90072616E736D697420666C61670A00FF1C1C
:101EE900B9FF1CBEFF1CC6FF1CD0FF1CD8FF1CE19C
:101EF9000008040C020A060E0109050D030B070F61
:101F090000010100010000010100000100010100C0
:081F190001020407080B0D0E84
:10400B0052668D0000000000000000000000000060
:05401B000000000000A0
:0100320022AB
:023D09008F57D2
:103D0B00906AA7E0FF04F074A92FF582E43466F5FE
:103D1B00837420F0E4FFEFC39D503BE55775F00330
:103D2B00A424E7F582E4341EF583E493FB7401933A
:103D3B00FA740293F98F82758300121A2CFE906A23
:103D4B00A7E024A9F582E43466F583EEF00F906AC0
:063D5B00A7E004F080C0A7
:013D6100223F
:103F5900742D2FF582E43461F583E0FE6420601648
:103F6900906AA7E0FD04F074A92DF582E43466F5A2
:063F790083EEF00F80DA78
:013F7F00221F
:10248000E4906AA7F0F54FE54F75F003A424E7F553
:1024900082E4341EF583E493FB740193FA7402938F
:1024A000F9121A13700302260EE4F551F552F55095
:1024B000742D2550F582E43461F583E0FF7003024A
:1024C0002609E54F75F003A424E7F582E4341EF5F0
:1024D00083E493FB740193FA740293F98551827536
:1024E0008300121A2CFEEFB5060875520105510241
:1024F0002604E5527003022604EE60030225FFADB8
:1025000051AF4F123D09E54F1470030225C11470FD
:10251000030225C51470030225C91470030225CFD8
:1025200024046003022609AF50123F59742D255030
:10253000F9E43461FA7B01C0031B8B5A755B0075AB
:102540005C00E4F55DD0031222DC8F568E558D546D
:102550008C53E4FFFEFDFCAB56AA55A954A853C307
:10256000121B696022AB56AA55A954A853E47F20D8
:102570007E1CFDFC121AC9121B5B906CAAEEF0A324
:10258000EFF0E4906CA9F0E47FB07E04FDFCAB5664
:10259000AA55A954A853D3121B69406D906CA97415
:1025A00001F0AB56AA55A954A8537F007EC2FD7C0A
:1025B00000121AC9121B5B906CAAEEF0A3EFF08018
:1025C00048D2068044D2048040D206D204803AAF7A
:1025D00050123F59742D2550F9E43461FA7B01C043
:1025E000031B8B5A755B00755C00E4F55DD003122C
:1025F00022DC8F568E558D548C5385567D800AE48F
:0E260000F552F55105500224B0054F02248713
:01260E0022A9
:102EF7007BFF7A1C79E2121719906CA9E0602FA367
:102F0700E0FEA3E0FFC3E49FFFE49EFEAB07FAE405
:102F1700F9F8FF7EC27D01FC121AC98F598E588DB0
:102F2700578C567BFF7A1D7904121719802F906CE6
:102F3700AAE0FEA3E0FFC3E49FFFE49EFEAB07FA0F
:102F4700E4F9F87F207E1CFDFC121AC98F598E58B0
:102F57008D578C567BFF7A1D79041217197BFF7AE0
:102F67001D7942A206E433F5561217197BFF7A1D25
:102F77007961A204E433F5561217197BFF7A1D799C
:102F870082A20AE433F556121719300A1F7BFF7A1B
:102F97001D79AC9066A1E075F00AA4FFAEF0E48F4E
:102FA700598E58F557F556121719801D7BFF7A1D54
:102FB70079D59066A1E075F00AA4FFAEF0E48F59C9
:102FC7008E58F557F5561217197BFF7A1E7900129E
:102FD70017197BFF7A1E7938E4857D59F558F5571F
:062FE700F5561217192235
:102BB0007E1E7F5F123854EF4E70037F01227E1E0F
:102BC0007F62123854EF4E7003022C57123BF6907E
:102BD0006CBC121B8DE4FFFEFDFC906CBCE0F8A306
:102BE000E0F9A3E0FAA3E0FBC3121B696025906C37
:102BF000BCE0F8A3E0A3E0A3E0E47F207E1CFDFCA2
:102C0000121AC9121B5B906CAAEEF0A3EFF0E490CD
:102C10006CA9F0E47FB07E04FDFC906CBCE0F8A3EE
:102C2000E0F9A3E0FAA3E0FBD3121B694038906CF3
:102C3000A97401F0906CBCE0F8A3E0A3E0A3E07FEE
:102C4000007EC27D017C00121AC9121B5B906CAA27
:102C5000EEF0A3EFF0800F906CAA74FFF0A374B8AD
:102C6000F0E4906CA9F07E1E7F68123854EF4E603D
:102C70000C124021EF24D024FF92068002C2067E6F
:102C80001E7F6E123854EF4E600C124021EF24D09C
:102C900024FF92048002C2047E1E7F74123854EF17
:102CA0004E600C124021EF24D024FF920A8002C211
:102CB0000A7E1E7F7A123854EF4E6013123BF6E400
:102CC0007B0AFAF9F8121AC99066A1EFF08005E4C0
:102CD0009066A1F07E1E7F80123854EF4E6007127E
:0B2CE0003BF68F7D8003757D027F00B6
:012CEB0022C6
:103B3500300E5D30102FC210E4906475F0906CA8C3
:103B4500E004FF906476F090667AE0906477F0A3E5
:103B55007410F09067AA63A20190647963A20112C0
:103B65001FFC7F0122E4906475F0A3E579F090666F
:103B75007AE0906477F0A37403F09069A163A201E1
:103B850090647963A201AF79121FFCC20E7F0122F6
:033B95007F00228C
:0234E4008F4E09
:1034E600906378E06410702A7F7975836305826340
:1034F600A2019068A763A201E54E24FCFF121FFCFF
:10350600D201E54E24FCF576E4F57BF56D7574FE87
:103516008073E54E24FCFFC313F54E754F04E4F5A6
:1035260050E550C3954E505DAF4F054F74752FF55E
:1035360082E43463F583E075F002A424A8F9746A82
:1035460035F0FA9068A47401F0A3EAF0A3E9F090CC
:1035560068A4E0FBA3E0FAA3E0F97440121A59AF9D
:103566004F054F74752FF582E43463F583E0FF90C1
:1035760068A4E0FBA3E0FAA3E0F9900001EF121AB9
:073586006B0550809CD20D83
:01358D00221B
:103ACA00906CAA74FFF0A374B8F0E4906CA9F0901B
:103ADA006AA7F0D22AF540F53FF53EF53DF54B755C
:103AEA004A66754996754899C203C208C20EC20C45
:103AFA00C20D757D02122BB0EF6003122480E4F52B
:103B0A004EE54E75F002A424A8F9746A35F0FA7BE2
:103B1A00019068A4EBF0A3EAF0A3E9F0E4121A59C1
:0A3B2A00054EE54EB4FADA123B989E
:013B3400226E
:103D6200C203D208C20ED22AE4F540F53FF53EF571
:103D72003DF54B754A6675499675489990668F125E
:103D82001B9900000000906693121B99000000002E
:103D9200906697121B990000000090669B121B9977
:093DA20000000000123E358F4EB6
:013DAB0022F5
:10329100E4FF0F2405F582E43461F5837408F00F2F
:1032A10074052401F582E43461F583E4F0754E017F
:1032B100754F66755092FEAB4EE5501550AA4F7092
:1032C10002154FF9121A13FDAC070F74052CF58284
:1032D100E43461F583EDF00EBE04DC754E01754FEB
:1032E10066755096E4FEAB4EE5501550AA4F70023C
:1032F100154FF9121A13FDAC070F74052CF582E472
:103301003461F583EDF00EBE04DC754E01754F6638
:1033110075509AE4FEAB4EE5501550AA4F70021558
:103321004FF9121A13FDAC070F74052CF582E43422
:1033310061F583EDF00EBE04DC754E01754F6675C7
:10334100509EE4FEAB4EE5501550AA4F7002154F4A
:10335100F9121A13FDAC070F74052CF582E43461E0
:08336100F583EDF00EBE04DC63
:013369002241
:082907008D4E8B4F8A5089515F
:10290F00E4F552EF54E0FEC4135407901F1993FEE1
:10291F00C454F04252EF541CFE1313543F934252CF
:10292F000551E5517002055014F9E552121A59E597
:10293F005254C0FEC4540F901F0993FEE552540C1D
:10294F0093FDEE2DF553E55254A0FEC4540F93FEA4
:10295F00E552540A93FDEE2DF554E4F552EF54036E
:10296F0025E0FFE433FEE54E5480FDC413131354EA
:10297F0001FDEEEF4D2419F582741F3EF583E493AC
:10298F00FFC454F04252E54E5470FFC4540F901FD1
:10299F0019934252AB4F0551E551AA5070020550A1
:1029AF0014F9E552121A59E55254C0FFC4540F904E
:1029BF001F0993FFE552540C93FEEF2E2553F55349
:1029CF00E55254A0FFC4540F93FFE552540A93FEEF
:1029DF00EF2E2554F554E4F552E54E540EFFC31374
:1029EF00901F1993FFC454F04252E54E5401FF3328
:1029FF00333354F84252E5525408FFC313901F0962
:102A0F0093FFE55254C0FEC4540F932F042553F582
:102A1F0053E55254A0FEC4540F932F042554F5547C
:102A2F00E5535401FF25E025E04252E5545401FFE0
:102A3F0025E04252E552540EFFC313901F199342E3
:102A4F0052AB4F0551E551AA507002055014F9E5EC
:042A5F0052121A599C
:012A63002250
:102A640030014FE56D704B74A7257BF582E4346823
:102A7400F583E0FD7B017A6A79A1AF7412290775A9
:102A840074FF857D6D057BD57602C201906693E067
:102A9400FCA3E0FDA3E0FEA3E0FFE4FAF9F8EF24D1
:102AA40001FFEA3EFEE93DFDE83CFC906693121B03
:102AB4008D22200503300F493005117B017A6A7994
:102AC400A17DFF7FFB122907C205800F7B017A6A73
:102AD40079A17DFE7FFB122907C20F906693E0FC6B
:102AE400A3E0FDA3E0FEA3E0FFE4FAF9F8EF24017C
:102AF400FFEA3EFEE93DFDE83CFC906693121B8D27
:102B0400229066A2E0FF04F0EF75F002A424A8F975
:102B1400746A35F0FA9068A47401F0A3EAF0A3E9AA
:102B2400F09068A4E0FBA3E0FAA3E0F9121A1320E2
:102B3400E6099066A2E0C394FB40C69066A2E0FF5B
:102B4400B4FB17E4F0E56D6002156D906AA174EEB4
:102B5400F0A37447F0A37414F022EF14FF90000163
:102B6400121A2CFD7B017A6A79A11229079068A4B4
:102B7400E0FBA3E0FAA3E0F9121A1354BF121A59A6
:102B8400E56D6002156D906693E0FCA3E0FDA3E0A3
:102B9400FEA3E0FFE4FAF9F8EF2401FFEA3EFEE9C0
:0C2BA4003DFDE83CFC906693121B8D2266
:1013380030072DC3E5279547FFE5269546FED3EFF1
:101348009440EE940040197B087D40AF47AE4612AA
:1013580031B6E5472440FFE43546540FF5468F473C
:101368002003030215CFE5435438653A602C906793
:10137800A9E064036024E53A24085438F53A1313C5
:1013880013541F242AF8E6FFE0FE04F074A42EF597
:1013980082E4346AF583EFF080CC9067A9E06403B7
:1013A8006003021604F0906AA4E064EE701EA3E0E5
:1013B800B44719A3E0B41414201E030215B37E1E0B
:1013C8007F86E4FBFDFC122CEC0215B3301E0D7E6B
:1013D8001E7F8F7C6A7DA47B03122CECE49066A3AD
:1013E800F090669FF0906AA4E0FF54E0FE9066A338
:1013F800F0EF540EFF25E04EFFF0906AA5E0FE5492
:10140800C0FDC4131354034FFF9066A3F0EE54209D
:10141800FE25E025E0FE90669FF0906AA5E0540E58
:10142800FD33333354F84EFE90669FF0906AA6E081
:10143800FD54E0FCC4540F4EFE90669FF0ED540836
:10144800FD131313541F4EFEF0FD7B017A6679A637
:101458001229079066A6E0FF906AA4E0B5071890E5
:1014680066A7E0FF906AA5E0B5070C9066A8E0FFC4
:10147800906AA6E06F6038201C0D7E1E7F997C6AFA
:101488007DA47B03122CEC906697E0FCA3E0FDA3FF
:10149800E0FEA3E0FFE4FAF9F8EF2401FFEA3EFEDC
:1014A800E93DFDE83CFC906697121B8D0215B39050
:1014B800668FE0FCA3E0FDA3E0FEA3E0FFE4FAF9F9
:1014C800F8EF2401FFEA3EFEE93DFDE83CFC9066AA
:1014D8008F121B8D9066A3E0FF2402605514607084
:1014E8008000EFC394F940030215B3AE790579740F
:1014F800A12EF582E43469F583EFF090669FE0FF52
:10150800AE79057974A12EF582E43469F583EFF09C
:10151800301C030215B37E1E7FA5122FED749F2584
:1015280079F582E43469AF82FEE4FB7D021231B6BC
:10153800807990669FE0FF6017300B02D20FD20BC4
:101548009066A4EFF0E49066A0F0906CA8F0805B41
:10155800300B589066A4E0603C90669FE0FF906C6A
:10156800A8E0FE04F074AA2EF582E43467F583EF50
:10157800F09066A0E02FF09066A4E014F0201C2BF9
:101588007E1E7FAF122FED90669FE0FF7E007D02EA
:101598001230D58016C20B90669FE0FFA3E0B50716
:1015A80008D20ED205D2108002D20F0570E5706401
:1015B8001F7049C203F540F53FF53EF53DD22AE5D7
:1015C800796039D20E8035202A32C20EE49067A99C
:1015D800F0D203F579F570201C227E1E7FB9122FF8
:1015E800EDAF40AE3FAD3EAC3D7810121B7A7D03A7
:1015F8001230D5AE3FAF407D031230D5200C030228
:10160800168BE54424085438FFE53B54386F6004D2
:101618007E0180027E00E57A640360047D01800219
:101628007D00EE5D601F74A1257AF582E4346AF5C9
:1016380083E0FEE544131313541F2432F8A6068FE3
:1016480044057A80BDE57A640370630573E573B475
:101658002005C20CD20822E4F57A122A64201C4E16
:101668007E1E7FCA122FEDAF737E007D021230D529
:101678007E1E7FD5122FED7E6A7FA1E4FB7D0312CB
:1016880031B622E4F57A906AA17466F0A37496F0F4
:10169800A37499F0201C127E1E7FD7122FED7E6A4C
:0E16A8007FA1E4FB7D031231B6D20CE4F57392
:0116B6002211
:0B408C00300D05C20D7F01227F0022D5
:03409E00C2AE228D
:1036C6000208A7E493A3F8E493A34003F68001F26B
:1036D60008DFF48029E493A3F85407240CC8C33305
:1036E600C4540F4420C8834004F456800146F6DFD4
:1036F600E4800B0102040810204080904005E47E1F
:10370600019360BCA3FF543F30E509541FFEE493C8
:10371600A360010ECF54C025E060A840B8E493A38F
:10372600FAE493A3F8E493A3C8C582C8CAC583CABA
:10373600F0A3C8C582C8CAC583CADFE9DEE780BE72
:01402000009F
:101A1300BB010689828A83E0225002E722BBFE02D1
:091A2300E32289828A83E4932204
:101A2C00BB010CE58229F582E5833AF583E022506F
:101A3C0006E92582F8E622BBFE06E92582F8E222B9
:0D1A4C00E58229F582E5833AF583E49322D3
:101A5900BB010689828A83F0225002F722BBFE016C
:021A6900F32266
:101A6B00F8BB010DE58229F582E5833AF583E8F0B1
:101A7B00225006E92582C8F622BBFE05E92582C85D
:021A8B00F22245
:101A8D0075F008758200EF2FFFEE33FECD33CDCC10
:101A9D0033CCC58233C5829BED9AEC99E582984093
:101AAD000CF582EE9BFEED9AFDEC99FC0FD5F0D670
:101ABD00E4CEFBE4CDFAE4CCF9A88222B800C1B99A
:101ACD000059BA002DEC8BF084CFCECDFCE5F0CBD8
:101ADD00F97818EF2FFFEE33FEED33FDEC33FCEB11
:101AED0033FB10D703994004EB99FB0FD8E5E4F9CC
:101AFD00FA227818EF2FFFEE33FEED33FDEC33FCB9
:101B0D00C933C910D7059BE99A4007EC9BFCE99AAC
:101B1D00F90FD8E0E4C9FAE4CCFB2275F010EF2FF1
:101B2D00FFEE33FEED33FDCC33CCC833C810D707F1
:101B3D009BEC9AE899400AED9BFDEC9AFCE899F82C
:0E1B4D000FD5F0DAE4CDFBE4CCFAE4C8F922BF
:0E1B5B00C3E49FFFE49EFEE49DFDE49CFC229B
:101B6900EB9FF5F0EA9E42F0E99D42F0E89C45F0D2
:011B79002249
:101B7A00E8600FECC313FCED13FDEE13FEEF13FF49
:031B8A00D8F1226D
:0C1B8D00ECF0A3EDF0A3EEF0A3EFF022CB
:101B9900A8828583F0D083D082121BB0121BB012A9
:101BA9001BB0121BB0E473E493A3C583C5F0C583CE
:101BB900C8C582C8F0A3C583C5F0C583C8C582C896
:011BC90022F9
:1016B700E5622456F8E60562227853302802785608
:1016C700E475F001121C19021A132021EB7F2ED2A8
:1016D700218018EF540F2490D43440D4FF30250BC9
:1016E700EF24BFB41A0050032461FFE563600215BD
:1016F700630566E5667002056530280D7853E47565
:10170700F001121C19EF021A59023DAC7403D228DA
:101717008003E4C228F5628B538A548955E4F56344
:10172700F565F566E56360077F201216F280F575AB
:1017370064FFC222C221C223C224C226C227C229F1
:101747001216C0FF700D3028057F00121703AF6611
:10175700AE6522B4255FC2D5C2251216C0FF24D0BC
:10176700B40A00501A75F00A786330D50508B6FF39
:101777000106C6A426F620D5047002D22480D924F7
:10178700CFB41A00EF5004C2E5D225021903D222C2
:1017970080C6D22180C0D22380BCD2D580BAD226BF
:1017A70080B47F201216F22023077401B56300402E
:1017B700F11216B7FF1216F202172BD229D2278081
:1017C700951216B7FB1216B7FA1216B7F94A4B70ED
:1017D7000679D47A197BFF20232EE563602A7E00E1
:1017E7008E82758300121A2C60060EEE656470F007
:1017F700C2D5EBC0E0EAC0E0E9C0E0EE12194AD07A
:10180700E0F9D0E0FAD0E0FB121A13FF60AAEBC0B0
:10181700E0EAC0E0E9C0E01216F2D0E02401F9D016
:10182700E03400FAD0E0FBE5640460DCD564D980DD
:10183700877BFF7A197946D223809C7910800279B9
:1018470008C227C2298008D2D5790A8004790AC23A
:10185700D5E564047002F564E4FAFDFEFF1216B7DD
:10186700FC7B082022131216B7FD7B1030210A12C9
:1018770016B7FE1216B7FF7B20EC3382D592D550F0
:1018870013C3E43021069FFFE49EFEE42022039D5C
:10189700FDE49CFCE4CBF8C222EC700CCFCECDCC9F
:1018A700E824F8F870F38017C3EF33FFEE33FEED4B
:1018B70033FDEC33FCEB33FB994002FB0FD8E9EB2C
:1018C700302205F8D0E0C448B222C0E00AEC4D4E01
:1018D7004F78207B0070C2EAB5640040BCC0E012BC
:1018E700194CD0F0D0E0202204C4C0E0C4B222C01A
:1018F700F01216DBD0F0D5F0EB02172B121C78177D
:10190700C85318425817994C17954218464F184E06
:0F19170044184E4917AE4318545518384618381F
:101926004518384719F450179D2D17A12E17C42BAB
:1019360017A52317C22019DD2A175D48000017BC1A
:101946003F3F3F00790AA2D5202414302609B9105A
:10195600020404B9080104A2D5202702500104207C
:1019660023689223B563005034C0E07F20302419E9
:101976007F30A22372277226500F1219A3C223C2E8
:1019860027C226C2297F30800F302603E9C0E01225
:1019960016F2302603D0E0F9D0E0B563CC30261736
:1019A6007F30B9100C1216F27F583025077F7880E9
:1019B60003B908031216F23023057F2D0216F27FB3
:1019C600202029F87F2B2027F322922380CF286E10
:1019D600756C6C2900D2221216B73022F8C2227812
:1019E6006330D50108F602175D2D5043495812168B
:1019F600B72403B405004001E49019EF931216E3EF
:0D1A0600743A1216E3D224756304021842EC
:1022DC008B578A588959E4F563F562F561F560F519
:1022EC005EF55FE55B455C455A6012EBC0E0EAC009
:1022FC00E0E9C0E0AB5AAA5BA95C121C29AB5705FC
:10230C0059E559AA587002055814F9121A13F564B4
:10231C00C394094007E564D3940D40E1E56464205F
:10232C0060DBE564B42D05435F038016E564B42BD4
:10233C0005435F01800C74FF2559F55974FF35581E
:10234C00F558E55D60046410703FAB57AA58A95965
:10235C00121A1364306009E55D702E755D0A8029D0
:10236C00900001121A2CFF64786004EFB4581343E8
:10237C005F01755D1074022559F559E43558F5580F
:10238C008007E55D7003755D08AB570559E559AAE3
:10239C00587002055814F9121A13F564C39461406D
:1023AC000AE564D3947A50035364DF74D02564F542
:1023BC0064C3940A400CE5649411406D74F925646F
:1023CC00F564E564D3955D5060435F018563688572
:1023DC006267856166856065AF5D7E00E4FCFDAB80
:1023EC0063AA62A961A860121BCAC8ECC8C9EDC96E
:1023FC00CAEECACBEFCBE4FCFDFEEB2564F563EE35
:10240C003AF562ED39F561EC38F560AF63AE62AD6B
:10241C0061FCAB68AA67A966A865D3121B69500357
:10242C00022395435F04022395E55F20E003E480DB
:10243C002DE55B455C455A601EAB57E55924FFF909
:10244C00E55834FFFAEBC0E0EAC0E0E9C0E0AB5A73
:10245C00AA5BA95C121C29E55F30E20774FFFFFE42
:10246C00FDFC22E55FAF63AE62AD61AC6030E103B1
:04247C00021B5B22C2
:101BCA00E88FF0A4CC8BF0A42CFCE98EF0A42CFCBA
:101BDA008AF0EDA42CFCEA8EF0A4CDA8F08BF0A438
:101BEA002DCC3825F0FDE98FF0A42CCD35F0FCEB97
:101BFA008EF0A4FEA9F0EB8FF0A4CFC5F02ECD395C
:0F1C0A00FEE43CFCEAA42DCE35F0FDE43CFC22C8
:101C1900FAE6FB0808E6F925F0F618E6CA3AF622CC
:101C2900BB011A89828A83D0F0D0E0F8D0E0F9D0DC
:101C3900E0FAD0E0FBE8C0E0C0F0021CA75016E9CA
:101C4900F8D083D082D0E0F9D0E0FAD0E0FBC082AE
:101C5900C083021C9EBBFE16E9F8D083D082D0E077
:0F1C6900F9D0E0FAD0E0FBC082C083021CB022A9
:101C7800D083D082F8E4937012740193700DA3A3FB
:101C880093F8740193F5828883E47374029368600F
:061C9800EFA3A3A380DF0F
:091C9E00EBF608EAF608E9F6226B
:091CA700EBF0A3EAF0A3E9F0223E
:091CB000EBF208EAF208E9F22265
:00000001FF
